:1000000002004E022003000000000002200B00004E
:10001000000000022013000000000002201B00006E
:10002000000000022023000000000002202B00003E
:10003000000000022033000000000002203B00000E
:10004000000000022043000000000002204B43AFEC
:10005000019006C074FFF0759E85759D08759852D5
:1000600075985AC2983098FDE599B411F602037D4F
:10007000A29822A29922E59922F59922C29922D228
:100080009922C29822C2AC22D2AC222222C0E0C065
:1000900082C083C006C007AE83AF829006C0E0B4C2
:1000A000FF35C001C002C003EEF0A3EF53E0C0F083
:1000B000FF900680AB82AA8379408E838F82E4937F
:1000C000A3AE83AF828A838B82F0A3AA83AB82D94B
:1000D000E9D003D002D001D007D006D083D082D09F
:1000E000E022C083C082C0E0E582543F90068025B4
:1000F00082F582D0E0F0D3D082D08322C083C08248
:10010000C0009006C0E0F5C7A3E0F5C675B9F0756C
:10011000B9059006807840E0F5BC75B982A305C6A4
:10012000D8F575B90F9006C074FFF0D000D082D01A
:100130008322C0E012008D1200E21200FCD0E02207
:1002000000000000000000000000000000000000EE
:1002100000000000000000000000000000000000DE
:1002200000000000000000000000000000000000CE
:1002300000000000000000000000000000000000BE
:1002400000000000000000000000000000000000AE
:10025000000000000000000000000000000000009E
:10026000000000000000000000000000000000008E
:10027000000000000000000000000000000000007E
:10028000000000000000000000000000000000006E
:10029000000000000000000000000000000000005E
:1002A000000000000000000000000000000000004E
:1002B000000000000000000000000000000000003E
:1002C000000000000000000000000000000000002E
:1002D000000000000000000000000000000000001E
:1002E000000000000000000000000000000000000E
:1002F00000000000000000000000000000000000FE
:10030000C082C083900709F0E5D0A3F0E4F5D0C522
:10031000A8A3F0D0E0A3F0D0E0A3F0D0E0A3F0D009
:10032000E0A3F0A3E0C581F0E5F0A3F0E8A3F07846
:100330000008A3E0C6F0E8B46FF712008C120E803C
:10034000120AFA1209FF1209ED1209ED1209ED1253
:0E03500009FF90070EE8F0A3E9F012007F22EB
:1003670056342E303000000021100007C40700204B
:10037700230040004000758107900709E47805F0E5
:10038700A3D8FC7420F0A37400F0A37407F0A3E4CF
:10039700F0F52304F524900701790078A51203FAF4
:1003A70078331203FA78CC1203FAE960107A0B7DDE
:1003B70000120AACE4F530F531900708F0120E8010
:1003C7001207B2B4110AE5231207A6F4F52380F049
:1003D700B40107E5241207A680E61203E680E1F5DB
:1003E700251414540E9007E2FF93CFA3938F83F540
:1003F70082E473E06849F9E8F0A32274061207A6BD
:10040700E5281207A69007047804E01207A6A3D8E8
:10041700F974041207A6227528001207BEF5266094
:10042700371207BEF5831207BEF5821207BEF527FE
:10043700AF26BF050312008D1207BE1208C4A3D54D
:1004470027F61207BEAF26BF05031200FCE525609D
:1004570003752802120402221207BE90070EF0A3AA
:100467001207BEF01207BE80D97528001207BEF525
:10047700261207BEF5831207BEF5821207BEF527BF
:100487001207BEE5256007752802120402227525AA
:100497000074021207D2E52660121209661207D20B
:1004A700A3D527F6E4C395251207D22290070EE0BD
:1004B7001207D2A3E01207D280EA7528001207BEFE
:1004C700F5291207BEF5271207BEF5261207BEF556
:1004D700831207BEF5821207BEE52560077528025D
:1004E70012040222E4B52906120A7B02040204B5AB
:1004F7002906120A9F02040204B52906120A9B0262
:10050700040204B52906120AA3020402120AD00241
:1005170004027528001207BEF5291207BEF5271237
:1005270007BEF5261207BEF5831207BEF58212072E
:10053700BEFA1207BEF81207BEF91207BEE525601C
:100547000775280212040222E4B5290C120BF112D6
:10055700007050031207B22204B52903020586046E
:10056700B52908C211120BB5020586C212120BB3C8
:1005770020120B12040212007050031207B22275E8
:10058700250074021207D27526047583007582E070
:100597001209661207D27582F01209661207D27520
:1005A70082D0752A081209665418F5821209661254
:1005B70007D2A3D52AF67582831209661207D27568
:1005C70082821209661207D290070EE01207D2A3A1
:1005D700E01207D27582D01209661207D2E4120719
:1005E700D2E41207D2E41207D2E41207D27582814D
:1005F700120966F5821207D27526011209661207DB
:10060700D21582D527F5E4C395251207D22275287E
:10061700001207BEF5261207BEF5831207BEF58244
:100627001207BE04F5291207BE04F5271207BEF507
:100637002A8006E52A1208C4A3D527F7D529F4127C
:1006470007BEE525600375280212040222752800FB
:100657001207BEE525600775280212040222C2119F
:10066700120BB590070EE0F8A3E0F9900704E8F045
:10067700A3E9F08883898275260512096690070623
:10068700F0120402227528001207BEF5291207BED0
:10069700F5271207BEE5256006752802020402E465
:1006A700B529065324FB02040204B5290643240492
:1006B70002040204B52908E4F530F5310204028585
:1006C7003082E5276009C3E5309527F5825007E5B5
:1006D70031700302040275250074021207D2758374
:1006E700F3E01207D20583E01207D20583E0120771
:1006F700D20583E01207D20583E01207D20583E013
:100707001207D20583E01207D20583E01207D2054C
:1007170083E01207D20583E01207D20583E01207B0
:10072700D20583E01207D20583E01207D20583E0E2
:100737001207D20583E01207D20583E01207D2051C
:1007470083E01207D20583E01207D20583E0120780
:10075700D20583E01207D2E4C395251207D222758A
:1007670028001207BEF5291207BEE5256006752881
:1007770002020402E4B52907900708F00204020404
:10078700B52907900708F002040290070474FFF0E8
:10079700A37403F0A37467F0A37416F002040212A3
:1007A700007350FB12007C1200792212007050FB7C
:1007B7001200761200822212007050FB120076128D
:1007C7000082C0E02525F525D0E02212007350FBFA
:1007D70012007C1200792525F52522041E047004D9
:1007E700C1051906150654068C0766900023E49385
:1007F7006402600B7402120132E49364027032A344
:10080700E49364086011E4936408600B74081201B0
:1008170032E4936408701AA3E49364936011E49339
:100827006477600B7493120132E49364937002C38C
:1008370022D32212008512007FE58124FAC886831D
:10084700088682A3A3A3A68218A683C8D0D0D08384
:10085700D082D0E01208610203003212007350FB0D
:1008670012007C12008890070BE0448045A8F02214
:10087700C0E0C082C083C0D075D000900708E07088
:1008870016D0D0D083D082D0E0022023C0E0C0822F
:10089700C083C0D075D00012007040030208B812A0
:1008A7000076120082B411030208B8B41B030208D1
:1008B7003A12007CD0D0D083D082D0E032AF26BFAE
:1008C7000102804DBF0202803DBF0302803ABF0490
:1008D70002803EBF05028009BF060280677528FFB8
:1008E70022C31200E2500422120132FFE493B5073B
:1008F7000122E528700F752803A882A983900706AF
:10090700E9F0A3E8F022F022A882F2220989827F87
:1009170001FEE582B47000400720E715F8EEF622E5
:10092700C082C0839007121209E3EEF0D083D08211
:1009370022BF010280E6C082C083F8EE120E9FD06C
:1009470083D082221392D51209D3C0E012099A0EDE
:10095700AF0613DFFDA2D533DEFDFED0E080B5AFD5
:1009670026BF0102802BBF0202801BBF0302801833
:10097700BF0402801CBF05028009BF0602804075C4
:1009870028FF22E49322E022A882E2228982197FAB
:1009970001E582B47000400620E716F8E622C0821F
:1009A700C0832412F582E43407F583E0D083D08234
:1009B70022BF010280E5C082C083120E9880ED122B
:1009C70009D312099A0E13DEFDE43322E582FE54A1
:1009D70007CE6E20E7050303032420222582F58234
:1009E700E43583F583220582D58202158315822299
:1009F700A3E0F8A3E0F9A322C8C583C8C9C582C983
:100A070022E0FB1209FFE493CB120A1A1209FFEB4B
:100A1700F0A3221208EFA322F528A882A983900742
:100A270004E527F0A3E526F0A3E9F0A3E8F022EA1E
:100A370075F006A490077C1209E3E0227A000A12F7
:100A47000A36B50002B322BA0AF422AE83AF827A1D
:100A57000A120A36601B1209F7C39FFBE89E700251
:100A67008009C3EF99FBEE98C37006BB02005001E3
:100A770022DADE22120A527404409D7800120A43D9
:100A8700740550941A8A277401F0A3EEF0A3EFF0CF
:100A9700E4020A1F7D0180067D0280027D00E527B2
:100AA700B480107A0A120A366002EDF0DAF722E80B
:100AB700020A1F7807B40A0050F5FA0A120A3678B4
:100AC7000660ECEDF0E4020A1FE5277807B40A0098
:100AD70050DD75F006A4FF9007822582F582E0F5C8
:100AE70027A3E0F8A3E0F9A3E0F52688838982E449
:100AF700020A1F90070E0209F8EC900F219354FC8D
:100B0700900B0B73020D9C00020B6F00020B690028
:100B1700020B6400020B5E00020B4C00020B480044
:100B2700020D8600020D8A00020EFA0074E0120E12
:100B370098F8A3A3A3E0F9A3E028F52CE439F52B53
:100B470022120B4C32120E96F9120993F52B120949
:100B570093F52CE9020E9D20111E120F0B8D2B8E83
:100B67002C22201113120F0BEC03C45407C52B546E
:100B7700F8452BF52B8D2C22AE2BAF2C7A0B120AB6
:100B870036120A8EE52454046003020B9C7A0B127A
:100B97000E42020DC4120402D212C2118003120CBB
:100BA700C5120BBE7A0A120CAB50F322D211E52400
:100BB70054046003120CC5120AFA882B892C1209F7
:100BC700FFE493FCA3E493FDA3E493FEEC900F21D1
:100BD700935403FA252CF52CE4352BF52B120B0037
:100BE700852C82852B8312034F22E526600BC000DC
:100BF700C00112034FD001D0001209FF7D00EA6047
:100C070005120A527D017A0B120A36ED120A90E597
:100C17002454046003020C37120E40E528600D646B
:100C2700037009120E80120402D21222120DC4227E
:100C3700120402533A00900708E07009120BB5122C
:100C47000CA950F822120070504F1207B2F8E53A7B
:100C5700053A600B14601414601814601C8037B8D0
:100C67001B0122B804301207A6802E88261207A679
:100C77008027883B1207A6802088821207A6853B1B
:100C870083E526700B90070EE01207A6A3E080030A
:100C97001209661207A6533A00120BB5120CA95097
:100CA700A4227A00120AFA0ABA0C0122120A36B4EE
:100CB70001F5A3E0B500F0A3E0B501EBB32290077F
:100CC70009E0F532A3E0F53390070CE0F534A3E033
:100CD700F535A3E0F536A3E0F537A3E0F538A3E053
:100CE700F539E53354182412F582E43407F583E027
:100CF700F8A3E0F9A3E0FAA3E0FBA3E0FCA3E0FD7F
:100D0700A3E0FEA3E0FF7583F3853082E532F005AB
:100D170083E539F00583E8F00583E9F00583EAF018
:100D27000583EBF00583ECF00583EDF00583EEF02A
:100D37000583EFF00583E535F00583E534F005839A
:100D4700E537F00583E536F00583E533F00583E500
:100D570038F00583E580F00583E590F00583E5A08D
:100D6700F00583E5B0F00530E530700375310122F9
:100D77007412120A1A7402120A1A7400020A1A8DDD
:100D8700067D037F00EE7E0330E7011F252CF52E3D
:100D9700EF352BF52D90035E12034F1209FF7804F0
:100DA700E6120A1A08DAF9120D7785822F120D77E3
:100DB700120DEBB52F06852E2C852D2B22900708BB
:100DC700E0601C1207F2500D120E807464F52812B1
:100DD7000402D21222120402D212120862800512F1
:100DE7000402D21212007C12008B900781786FE008
:100DF700C6F00582D5820215831582D8F2E0F890F5
:100E07000711E0F5F0900710E0C581F090070FE0BB
:100E1700C0E090070EE0C0E090070DE0C0E090074B
:100E27000CE0C0E090070BE0F5A890070AE09007F8
:100E370009F5D0E0D083D082227A01120AFAAE01F6
:100E4700AD00120A36B4012CC083C0821209F7C361
:100E5700EE99FCED98700CBC0200500775280874D9
:100E670001800C7412120A097402120A097403D061
:100E770082D083F00ABA0CCA227A0B120A36B4035C
:100E87000C7401F01209F7120A08120A08DAEC7456
:100E970081D210F880047881C210900709B8E00267
:100EA7008024A3B8D002801EA3B8A8028018A3B8D4
:100EB70083028012A3B88202800C900710B88102C7
:100EC7008004A3B8F007201002F022E02279E52081
:100ED70010027988C0E090035EE91208EFA982E565
:100EE70083C8A3120A1A7422120A1A89828883E411
:100EF700D0007374E0120E98852C82852B8393782B
:100F0700E0020E9F120E96C006F9E52C120913E5B2
:100F17002B120913E9D006020E9D01060F010102EB
:100F270001010101010101010101230A130101026C
:100F3700010101010101010101012306150102025D
:100F470001010101010101010101230A1901020245
:100F5700010101010101010101011E060203020253
:100F6700010101010101010101011E0A020302023F
:100F7700010101010101010101011E060203020233
:100F8700010101010101010101011E0A02290203F8
:100F9700020202020202020202021E0602250103E7
:100FA70002020202020202020202030A0201020212
:100FB7000101010101010101010102060201010113
:100FC70002020202020202020202020A02012323B1
:100FD700232323232323232323230206020101029E
:100FE70001010101010101010101020A02010123BD
:100FF70001011E1E1E1E1E1E1E1E010601010102EC
:1010070001010101010101010101010A01010102BF
:0A10170001010101010101010101C5
:00000001FF
